:100000000C941F030C9457030C9457030C94570340
:100010000C9457030C9457030C9457030C945703F8
:100020000C9457030C9457030C9432250C94ED2335
:100030000C9438270C9457030C9457030C945703D3
:100040000C9457030C9457030C9457030C945703C8
:100050000C9457030C94EB260C9457030C94570301
:100060000C9457030C9457030C9457030C945703A8
:100070000C9457030C9457030C9457030C94570398
:100080000C9457030C9457030C9457030C94570388
:100090000C9457030C9457030C9457030C94570378
:1000A0000C9457030C9457030C9457030509080943
:1000B0002D0945094B095609590959095909920A47
:1000C000920ADB09DD09E209080A2B0A2E0A310A25
:1000D000560A770A830A630DD70D6B0D350D390D5E
:1000E0006F0D3C0D720D7D0D470DCD0D4B0D810D2E
:1000F0004F0D850DAF0D530D890DB90D590D8F0D98
:10010000990D400D760D430D790D5E0D940DA50DE5
:10011000C50DC70D310D670DE00D090E0F0EFA0D5F
:10012000000E150E1B0E210ECA0ECA0EFC0EFC0E82
:10013000750F910FBA10BA10960F241035103510A4
:10014000FB1009110E11131118111D112211271185
:100150002C11311136113D11401143114611EA0C99
:10016000EA0CEA0CEA0CEA0CEA0C02222922D2235D
:100170002922D22375229822D2238D239D23000089
:10018000000000000000000000000000000000006F
:10019000000000000000000000000000000000005F
:1001A00000007E0F00D4FFFFFFC7000000780000B2
:1001B0000000000000002A2B2800000000000000C2
:1001C00000000000000000000029000000002C1EBC
:1001D0003420212224342627252E362D3738271E79
:1001E0001F202122232425263333362E37381F049F
:1001F00005060708090A0B0C0D0E0F101112131437
:1002000015161718191A1B1C1D2F3130232D3504F4
:1002100005060708090A0B0C0D0E0F101112131416
:1002200015161718191A1B1C1D2F3130354C0501D6
:100230000902A10185020901A10005091901290886
:100240001500250195087501810205010930093164
:100250001581257F95027508810609381581257F4E
:10026000950175088106050C0A38021581257F95D0
:100270000175088106C0C005010980A10185031927
:10028000012AB700150126B700950175108100C03D
:10029000050C0901A101850419012AA002150126F6
:1002A000A002950175108100C00660FF0961A101DF
:1002B0000962150026FF0095207508810209631563
:1002C0000026FF00952075089102C005010906A1CE
:1002D00001050719E029E715002501950875018139
:1002E000029501750881010507190029FF150026EF
:1002F000FF00950675088100050819012905950577
:1003000075019102950175039101C009025B00031B
:100310000100A0FA090400000103010100092111F4
:1003200001000122400007058103080001090401C2
:100330000002030000000921110100012222000730
:1003400005820320000107050303200001090402C0
:10035000000103000000092111010001227B0007B8
:100360000584032000011201000200000008756FDF
:1003700018550001010200011403730077006500A5
:1003800065007400310036007600320000001A0368
:100390003100750070006B006500790062006F002D
:1003A00061007200640073000000040309045F0030
:1003B0006000610056005C005D005E00570059005F
:1003C0005A005B00540021526200630058002078FC
:1003D00023782578277821782478267828782A7831
:1003E000297801000100010001000100007C0100EA
:1003F00001000100010001000100010001000100F5
:1004000001000100010001000100010001000100E4
:1004100001000100010001000100010001000100D4
:1004200001000100010001000100010001000100C4
:1004300001000100010001000100010001000100B4
:1004400001000100010001000100010001000100A4
:100450000100010001000100010001000100010094
:100460000100010001000100010001000100010084
:100470000100010001000100010001000100010074
:100480000100010001000100010001000100010064
:100490000100010001000100010001000100010054
:1004A0000100010001000100010001000100010044
:1004B0000100010001000100010001000100010034
:1004C0000100010001000100010001000100010024
:1004D0000100010001000100010001000100010014
:1004E0000100010001000100010001000100A9005C
:1004F000AA00A900AA0001000100010001000100FA
:1005000001000100010001000100010001000100E3
:1005100001000100010001000100010001000100D3
:1005200001000100010001000100010001000100C3
:1005300001000100010001000100010001000001B3
:100540000101010101010101020202020202020293
:100550000203030303030303030404040404040465
:100560000505050505060606060607070707070829
:10057000080808090909090A0A0A0B0B0B0C0C0CDC
:100580000D0D0D0E0E0E0F0F0F1010111111121276
:1005900013131414151516161717181819191A1AF3
:1005A0001B1B1C1D1D1E1E1F202021222223242454
:1005B000252626272829292A2B2C2D2D2E2F303190
:1005C0003232333435363738393A3B3C3D3E3F40A2
:1005D0004142434445464748494A4C4D4E4F50518D
:1005E0005354555658595A5B5D5E5F616264656647
:1005F00068696B6C6D6F7072737577787A7B7D7ECE
:100600008082838587888A8C8E8F91939596989A1D
:100610009C9EA0A2A3A5A7A9ABADAFB1B3B5B7BA35
:10062000BCBEC0C2C4C6C9CBCDCFD1D4D6D8DBDD09
:10063000DFE2E4E7E9EBEEF0F3F5F8FAFDFF112471
:100640001FBECFEFDAE0DEBFCDBF04B603FE18C099
:1006500080917C0390917D03A0917E03B0917F03F4
:100660008730904BA740B04B59F410927C03109206
:100670007D0310927E0310927F03E0E0F8E309957A
:1006800011E0A0E0B1E0EAE0FBE602C005900D92C7
:10069000AC3CB107D9F723E0ACECB1E001C01D924E
:1006A000AC37B207E1F70E9459030C9483350C94E0
:1006B0000000AFE4B0E0EFE5F3E00C94363585B729
:1006C000806885BF85B7806885BF84B7877F84BF12
:1006D0000FB6F894A89580916000886180936000BF
:1006E000109260000FBE90E080E80FB6F8948093FF
:1006F0006100909361000FBE88EE98E19093CD0168
:100700008093CC010E9431240E94D7248091E20082
:1007100084608093E20078948091AA028823A1F0FB
:100720001091E9001F709091EC00892F817090FD6D
:1007300080E8182B1092E9008091E80083FD0E9468
:100740001F211F701093E90082E084BD93E095BDE6
:100750009AEF97BD80936E000E940F32811102C004
:100760000E94FF3182E08093DF0142E351E0A0E389
:10077000B1E034E3E32E31E0F32E8D019A0161E024
:1007800070E0F90181919F01E82FE295EF70F0E0B0
:10079000D1A08F705B0102C0AA0CBB1C8A95E2F746
:1007A000C5019A2D90959D2191A392A1892B82A399
:1007B000F80181918F01E82FE295EF70F0E0D1A070
:1007C0008F705B0102C0AA0CBB1C8A95E2F7C501C1
:1007D0009A2D90959D2191A392A1892B82A3E21637
:1007E000F30679F68FE891E00197F1F700C0000079
:1007F0007091DF0100EE11E060E0671751F1FA013E
:100800002191AF01822F82958F7090E0FC0180A131
:1008100090E02F7002C0959587952A95E2F7817038
:100820009D91292F22952F7030E0F90120A130E011
:100830009F7002C0359527959A95E2F720FF02C078
:1008400092E001C090E0892BF80181938F016F5FE6
:10085000D4CF08E111E02CE1E22E21E0F22ED80104
:100860008D918D018F3F11F00E942D19E016F10638
:10087000B1F70CE111E090E2E92E91E0F92EF801D8
:1008800081918F018F3F11F00E942D19E016F10622
:10089000B1F784E0E3EEF1E0DF01A82E1D92AA9407
:1008A000E9F7EEECF1E0DF011D928A95E9F70E948D
:1008B000B51B811102C00E94C11B82E090E00E9422
:1008C00050348093D60184E090E00E945834909395
:1008D000D3018093D2010E944419BFEFE6E7F1E013
:1008E000B150E040F040E1F700C000000E94441920
:1008F0008091E30180FF08C06FEF7FEF80E090E020
:100900000E948C340E94C72683E090E00E945034FD
:1009100090E00E9499291092BE02E7EDF2E087EE86
:1009200092E02FEF3FEF219331938E179F07D9F776
:1009300010921103EAE2F3E08AE393E02FEF3FEF36
:10094000219331938E179F07D9F70E94B51B811110
:1009500004C00E94C11B0E94DF2E81E080933F03F0
:1009600046E050E06CE170E088EB92E00E94403499
:1009700010923F038091B8028C7F11F40E94DF2E09
:1009800084E091E09093EF028093EE028E010F5F7E
:100990001F4F8091AA02853009F063C0F0E4EF2E6A
:1009A000DD24D394A3E0CA2EB0E1FB2E8091AA02ED
:1009B000853009F050C08091AA02843009F439C012
:1009C0000E941C3380913E0381110DC00E94511181
:1009D000109213018091B8028370809312010E94DB
:1009E000F530C0921401D0923E031092F20288E1D9
:1009F000A82EB12C0FB6F894A895A09260000FBE57
:100A0000E092600083B7817F846083BF83B7816099
:100A100083BF7894889583B78E7F83BF0FB6F89491
:100A2000A8958091600088618093600010926000BA
:100A30000FBE8091A902882309F4B8CF0E944419FF
:100A4000E3EEF1E08191811176C527EE31E02E17BA
:100A50003F07C1F7ABCF0E94D5290E94D227109241
:100A60003E030E94441947ED51E021965FAF4EAF1F
:100A7000219783EE91E02C969FAF8EAF2C972BEDB4
:100A800031E0DC01FA0191918D9189272E173F0702
:100A900019F08823C1F322C0811120C00E942C27A5
:100AA0007C018091D4019091D501E816F90609F4F2
:100AB000B3C18FEF8DAB8EAB1FAA0E942C27816034
:100AC000782F99AF88AF4DA95EA96FA989AD0E9413
:100AD000DA0AF092D501E092D4019EC1ADE3B2E012
:100AE0002496BFAFAEAF2497E8E7F1E02696FFAFBC
:100AF000EEAF2697D12C2C96AEADBFAD2C974D9076
:100B00002C96BFAFAEAF2C972196EEADFFAD2197DF
:100B10003080342429963FAE2997332009F459C1F7
:100B200024966EAC7FAC249726962EAC3FAC2697CD
:100B3000C12C5524539429968FAD2997852109F40A
:100B400038C1852C8420CAAEDBAE81E0811001C0A3
:100B500080E08CAF0E942C278160782F9EAF8DAFF4
:100B60004AAD5BAD6CAD8EAD0E94DA0A882051F0C3
:100B7000D1018C918F3F31F02A968FAF2A9799241B
:100B8000939401C0912CE92CF12C80911103F70171
:100B9000E80FF11D3997ACF168E0A62EB12CAE1824
:100BA000BF08B7016F5F7F4F6F5E7C4FA50182E189
:100BB00093E00E947A35B701675F7F4F6F5E7C4F8D
:100BC000A5018AE193E00E947A35A501440F551FE3
:100BD000B701660F771F675E7F4F6F5E7C4F8AE2BB
:100BE00093E00E947A35B7016F5E7F4F6F5E7C4F56
:100BF000A50182E293E00E947A3588E0891980930A
:100C000011038091110390E02A96AFAC2A97AA2D88
:100C1000B0E09D01220F331F28573E4FAA0FBB1F84
:100C2000BD0167577E4F41E0480F9915C0F490E031
:100C3000FC01EF5EFC4FD9015C915183DB015C91BB
:100C400051872A96AFAC2A97A18A880F991FFC0179
:100C5000EF5EFC4F128E118E91E0842FE4CF8093D3
:100C60001103882009F4A5C08091B8028C7F8C37CD
:100C700009F09FC0D1018C918F3F09F49AC0E8E739
:100C8000F1E02896FFAFEEAF28977DE3872E72E064
:100C9000972E22961FAE229790E09C01220F331FC1
:100CA000A90148575E4F2E965FAF4EAF2E97D901E0
:100CB000A757BE4F6096BFAFAEAF60975401E12C0F
:100CC000F12C2896EEADFFAD2897EE0DFF1D80812B
:100CD0008F3F09F44DC02296BFAD2297BD110AC0C7
:100CE000CE1008C0F301208130E2230F08F42FEF6B
:100CF00020833EC090E02E96EEADFFAD2E97408152
:100D000050E0FC01EE0FFF1FE857FE4F2081421B11
:100D100051096096AEADBFAD60972C9130E0880F61
:100D2000991FFC01E858FE4F8189281B3109449F17
:100D3000B001459F700D700D1124229FC001239FAB
:100D4000900D900D1124860F971F0E94542F893209
:100D500078F438E2282F321B08F430E0313108F003
:100D600030E1D5012C91230F08F42FEFF5012083FA
:100D7000FFEFEF1AFF0A2FEFA21AB20A34E0E316D0
:100D8000F10409F09ECF22964FAD22974F5F229635
:100D90004FAF229754E0850E911C28968EAD9FADE3
:100DA0002897049628969FAF8EAF2897443009F075
:100DB00085CFC394550C9FEF291A390AAFEF6A1AF1
:100DC0007A0AB4E0CB12B7CE2196EEADFFAD2197F3
:100DD0004082D39421962EAD3FAD21972F5F3F4F98
:100DE00021963FAF2EAF219726964EAD5FAD269749
:100DF0004C5F5F4F26965FAF4EAF269724968EAD21
:100E00009FAD2497049624969FAF8EAF249794E0CD
:100E1000D91271CE0E9420270E941C33B12CA12C24
:100E20009DEF992E882483942CEF722E8091DF0100
:100E3000B81608F0AAC0CB2CD12CF601EE5CFE4F00
:100E40008081E82FE295EF70F0E0E0A1F0E08F7094
:100E500002C0F595E7958A95E2F7E170D601A05DAD
:100E6000BE4F8C91A82FA295AF70B0E090962C91B8
:100E700030E08F7002C0359527958A95E2F720FF04
:100E800002C092E001C090E08E2F892BD601A052C3
:100E9000BE4FEC912E2F237030E0482F082E000C0F
:100EA000550B2417350709F46EC0EE0FEE0FE82B33
:100EB000EC93EF70F0E0E05EFE4FD601A352BE4F20
:100EC0007D0190818C91890F8C93843034F1F601EF
:100ED000E552FE4F80818F5F80830E942C27BBA646
:100EE0007CA68DA68160782F9FA78EA74B2D5CEFE7
:100EF00061E08FA50E94DA0A0E942C27B8AA79AA7D
:100F00001AAA8160782F9CAB8BAB4B2D5CEF60E015
:100F10008CA90E94DA0A21E001C020E0F70180815B
:100F20008D3F2CF5F601E552FE4F80818150808384
:100F30000E942C27B9A29AA28BA28160782F9DA330
:100F40008CA34B2D5DEF61E08DA10E94DA0A0E9417
:100F50002C27BEA29FA218A68160782F9AA789A7E6
:100F60004B2D5DEF60E08AA50E94DA0A21E0D701EF
:100F70008C91082E000C990B64E070E00E941535EE
:100F8000F7018083A22AB39451CFA1100E94202799
:100F900086E0EBE0F3E0D80101900D928A95E1F74D
:100FA00010920D0310920E0310920F031092100373
:100FB0008B81811104C08C81882309F453C08091F6
:100FC000090390910A030E9411279C019091040348
:100FD000992309F4CFC22531310508F443C09F3F5E
:100FE00019F09F5F90930403FB80FF2061F00E9443
:100FF000A1301F1414F491E001C09FEF899F802D50
:10100000112480930D03FC80FF2061F00E94A13029
:101010001F1414F491E001C09FEF899F802D1124CB
:1010200080930E0330910D033323E1F020910E03E2
:101030002223C1F045EB3403C0011124992319F098
:1010400090930D0303C081E080930D0355EB2503BE
:10105000C0011124992319F090930E0303C081E07D
:1010600080930E038D81811104C08E81882309F441
:1010700053C080910703909108030E9411279C019F
:1010800090910503992309F47AC22135310508F4BA
:1010900043C09F3F19F09F5F90930503FD80FF20A1
:1010A00061F00E947F301F1414F491E001C09FEFA3
:1010B000899F802D112480930F03FE80FF2061F013
:1010C0000E947F301F1414F491E001C09FEF899FAC
:1010D000802D11248093100330910F033323E1F00E
:1010E000209110032223C1F045EB3403C0011124E9
:1010F000992319F090930F0303C081E080930F03AD
:1011000055EB2503C0011124992319F09093100386
:1011100003C081E08093100346E050E0B8018BE00B
:1011200093E00E946D35892BA9F480910D03811104
:101130000FC080910E0381110BC080910F038111AC
:1011400007C081E090911003911103C080E001C0BD
:1011500081E080FD0E94553086E0F801ABE0B3E00D
:1011600001900D928A95E1F70E94D2279091E201B9
:10117000891721F08093E2010E9420278091AA0222
:10118000843009F006CC83E08093E9008091E80088
:1011900082FFFFCB8091E80085FF21C00E94502490
:1011A00081111BC080E2C82ED12C780109C080912A
:1011B000F100D7018D937D01B1E0CB1AD10869F020
:1011C0008091E80085FDF3CF8091E8008B778093D4
:1011D000E8000E945024882399F391E001C090E038
:1011E0008091E8008B778093E800992309F4D1CBB4
:1011F0002981822F90E0FC013197E531F10508F05B
:1012000091C1EA5AFF4F0C9429351A828BE0D8C05D
:101210008A81823009F4A6C150F4813009F082C17C
:101220000E9420279B838C837D836E837DC18330C6
:1012300041F0843009F076C11B821C821D821E821F
:1012400073C18091E3018B838091E4018C83809151
:10125000E5018D838091E60154C18A81823061F07D
:10126000853009F05FC19091B80281E089278093B1
:10127000B8021092140158C16B817C818D819E81CE
:101280000E942F350E94DB314FC14C816B818A81D6
:101290000E94AD3135C12D813E813227232732276F
:1012A0004C816B818A810E9486313EC10E94582800
:1012B0003BC18A81833009F035C1283009F443C02D
:1012C000293009F46DC08B818230D1F070F4813007
:1012D00009F02AC14C812FEF429F412D11248091AA
:1012E000B90220E06091BA022AC0833021F1843033
:1012F00009F01AC18C8120E04091BB026D811FC0B2
:101300008C819091B802811109C0892F837011F0EE
:10131000109214019C7F9093B80206C1292F23706C
:1013200011F4109214019C7F91609093B80260E0D8
:101330000E94EC32F9C08C818093BC02F5C090E031
:101340000E948E32F1C08B818230E1F078F48130DE
:1013500009F0EAC08091BB02EFEF8E9FC00111241B
:101360006FEF70E00E9401356C83DEC08330A1F026
:10137000843009F0D9C08091B9028C838091BA027F
:101380008D83D2C08091B802982F937019F0869502
:10139000869504C080E002C08091BC028C83C4C0EA
:1013A00046E050E06CE170E088EB92E00E945E3431
:1013B00010923F03B9C080E152C082E08A838AE480
:1013C0008B83B2C0EA80FB80FE24EF24FE24CC8015
:1013D000D12C5801C7018A549E4F9501201B310B17
:1013E0002C153D0508F0A0C0FAE4EF16F2E0FF0668
:1013F00030F40E945034D50114968C9302C0F5014C
:101400001482FFEFEF1AFF0A2FEFA21AB20AE2CFFF
:10141000EA80FB80FE24EF24FE24CC80D12C5801EE
:10142000C7018A549E4F9501201B310B2C153D0599
:1014300008F07AC03AE4E31632E0F30628F4D50166
:1014400014966C910E946E34BFEFEB1AFB0AEFEF1B
:10145000AE1ABE0AE5CF0E94482866C08AE08A8399
:1014600063C0EA80FB80FE24EF24FE24CC80D12CD4
:101470005801C70186969501201B310B2C153D059F
:1014800008F052C0F0E4EF16F1E0FF0630F40E94DD
:101490005034D50114968C9302C0F5011482FFEFED
:1014A000EF1AFF0A2FEFA21AB20AE3CFEA80FB80FD
:1014B000FE24EF24FE24CC80D12C5801C70186964F
:1014C0009501201B310B2C153D0570F530E4E3161A
:1014D00031E0F30628F4D50114966C910E946E3425
:1014E000BFEFEB1AFB0AEFEFAE1ABE0AE7CF41E0FF
:1014F0008C81811101C040E06B818A810E944D3155
:101500009D838E8311C02D813E8132272327322770
:1015100041E08C81811101C040E06B818A810E9491
:101520001B3102C08FEF898340E250E0B80182E0B6
:101530000E9467262ECAF9BC82E189BD09B400FE6B
:10154000FDCF8091D8008F7D8093D8008091E000FE
:1015500082608093E0008091E00081FDFCCF0E94DA
:10156000D52924CA85E290E00E9450341B821C8257
:101570001D82C7CF2B30310508F033CD73CD2B3012
:10158000310508F088CDC8CD0E94D5292FEF84E31E
:101590009CE0215080409040E1F700C000009CE0BA
:1015A00088E10FB6F894A895809360000FBE9093E1
:1015B0006000FFCFA7E1B0E0E0EEFAE00C94453523
:1015C0004B8B5C8B6D8B7E8B8F8B61111092960297
:1015D00086E09E01235F3F4FD901E82F1D92EA95D7
:1015E000E9F795E0FE017396D90101900D929A9565
:1015F000E1F79C894E895F897B897D879E876F870C
:10160000598B488BF901DE01179601900D928A954E
:10161000E1F7CE0107960E94151D81113EC086E0BC
:10162000FE013796DE01119601900D928A95E1F741
:10163000FF81E8856A857B856115710531F0EF3F93
:1016400031F481E0FF3F19F403C081E001C080E084
:1016500080FD23C020915B0230E0C90101968770B4
:10166000992740918C0250E08417950779F1F9830E
:10167000EA837D836C8396E0929FD001939FB00DA7
:101680001124A45ABD4FFE01319601900D929A95F6
:10169000E1F780935B020E94A21C16E080918C020D
:1016A00090915B028917F9F0189FC0011124845AA8
:1016B0009D4F0E94151D8823B1F080918C0290E00F
:1016C00001968770992780938C02E8CF0E94D529D4
:1016D00010925B0210928C02E5E5F2E086E0DF01F9
:1016E0001D928A95E9F76796E3E00C946135ADE0C9
:1016F000B0E0EDE7FBE00C943635FC018081918190
:1017000023813481232B31F09F3F31F491E08F3FCF
:1017100019F403C091E001C090E090FDBEC57F01C7
:1017200085E0DE01199601900D928A95E1F7F701A7
:10173000228189859A85222349F00E94FE28182F4C
:10174000682F89859A850E94582903C00E943F29E5
:10175000182F69857A85812F0E94F7198C01F7016E
:101760008281882309F42CC1980122503747203107
:10177000310508F041C18FEF93E00E945034811190
:1017800029C1025036EBA32EBB24B394002379F079
:10179000A114F4E0BF0609F41DC1C5010E94503434
:1017A000811101C001502FEFA21AB20AEFCFCE0172
:1017B00001962C0188E0F20111928A95E9F72AE05E
:1017C000322E85010F5F1F4FC5010E94503489835F
:1017D0001A82882309F4FEC0813009F041C06501F6
:1017E000F2E0CF0ED11CC8010E9450348A838823B6
:1017F00009F4F0C09FEF980F933060F423E0A20E3D
:10180000B11CC6010E9450348B83882309F4E2C0C6
:101810001C8229C0843031F54E0133E0830E911CC7
:1018200002E010E056018FEFA81AB80AC6010E9424
:101830005034F40181934F01882309F4CBC08C37D5
:1018400041F4E2E0F0E0EC0FFD1FE00FF11F108229
:101850000AC00F5F1F4F65010730110519F7BAC0A5
:10186000580101C056018201F8012081222309F4A8
:10187000A8CF213009F04CC08181813049F4680142
:10188000F2E0CF0ED11CF80182810E94EE2B0AC03B
:10189000823051F46801F2E0CF0ED11CF801828150
:1018A0000E94492B860189C0833049F46801F2E027
:1018B000CF0ED11CF80182810E94E52AF3CF84303B
:1018C00019F00F5F1F4F79C0F80122810E5F1F4F83
:1018D00080E090E030E0205331092A30310568F48F
:1018E000389EA001399E500D1124C901840F951F07
:1018F0000F5F1F4FF8012081EDCF009709F45DC005
:10190000EFE9FFE03197F1F700C000000197F5CF54
:10191000E22FF0E0E255FE4F2490822F86958695C7
:10192000869590E0FC01E256FE4F64902770712C82
:10193000022E02C0759467940A94E2F7F1E06F22D8
:101940007724FC01E257FE4F8490912C022E02C0B6
:10195000959487940A94E2F731E083229924FC015C
:10196000E258FE4FC490D12C02C0D594C7942A955A
:10197000E2F781E0C822DD246114710419F081EEE0
:101980000E94492B8114910419F086EE0E94492B84
:10199000822D0E94EE2B8114910419F086EE0E9494
:1019A000E52A6114710419F081EE0E94E52AC11440
:1019B000D10419F08CE20E94EE2B0F5F1F4F54CF21
:1019C000011537E7130709F042C181E00E9477292A
:1019D0000E949C1E80918D02877009F45EC4F701FD
:1019E0008281882309F459C48091D30182FF55C4B0
:1019F00082E00E946E1C51C40115F7E71F0711F425
:101A000081E005C0013027E7120721F482E00E943F
:101A10008929DECFF801E851FC47E730F10508F4E9
:101A2000E5C0882309F45BC11092EB02C80190570E
:101A3000839708F013C184E090E00E94583490939B
:101A4000D3018093D201F801E150F047E232F10571
:101A500020F4E559FF4F0C9429358091D201816023
:101A6000ACC08091D3018860B4C08091D201826003
:101A7000A4C08091D20120C08091D20188609DC015
:101A80008091D3011EC08091D3018260A2C0809159
:101A9000D201806192C08091D20180628EC080911B
:101AA000D20180648AC00E94D5298091D2018068C9
:101AB00084C08091D201886084607FC08091D3010E
:101AC0008260816086C08091D2018E7F76C08091D5
:101AD000D301877F7EC08091D2018D7F6EC08091BF
:101AE000D20120C08091D201877F67C08091D3014D
:101AF0001EC08091D3018D7F6CC08091D2018F7EFA
:101B00005CC08091D2018F7D58C08091D2018F7BC3
:101B100054C00E94D5298091D2018F774EC0809108
:101B2000D201877F8B7F49C08091D3018D7F8E7FCB
:101B300050C08091D20182FB222720F991E09227A8
:101B400090FB82F990FB83F938C08091D301982FE4
:101B5000909591708E7F892B90FB81F93AC080918E
:101B6000D20186FB222720F991E0922790FB86F98B
:101B700024C00E94D5298091D20187FB222720F919
:101B800091E0922790FB87F918C061E001C060E006
:101B90008EE090E00E946E341EC08091D20184FBE2
:101BA000222720F991E0922790FB84F906C08091CA
:101BB000D201982F909590FB80F98093D2010BC0B1
:101BC0008091D30183FB222720F991E0922790FB9B
:101BD00083F98093D3016091D2017091D30184E0A5
:101BE00090E00E948C340E94D529F4CEE357FF4F39
:101BF0000C94293506E221EE41EE6AE17CE705C04E
:101C000007E225EE45EE6BE17CE7C7010E94DF2786
:101C1000E1CE06E221EE40EE68E17CE7F6CF07E296
:101C200025EE44EE69E17CE7F0CF06E221EE42EEDC
:101C30006CE17CE7EACF07E225EE46EE6DE17CE75A
:101C4000E4CF08E221E045EE6EE17CE7DECF013033
:101C500097E7190709F0DECE82E0B8CE0631ECE74F
:101C60001E0709F4A6C203309CE7190721F140F4CE
:101C70000115FCE71F0789F001301C4711F13EC038
:101C80000B353CE7130739F10C358CE71807D9F011
:101C90000A351C4799F581E01FC00E94D529EFEF56
:101CA000F4E32CE0E150F0402040E1F700C00000F8
:101CB0000E94C7268FCE6FEF7FEF80E090E00E94FA
:101CC0008C340E94C40A8091D30182FB882780F95A
:101CD00091E0892701C080E00E948B1C0FC0063173
:101CE000FCE71F0709F475C2809197028272F80120
:101CF000E052F847E531F10508F479C2F701828135
:101D000000811181882349F0C8010E94FE28D82E45
:101D1000682FC8010E94582904C0C8010E943F29A9
:101D2000D82EB8018D2D0E94F7190E94171A8C0128
:101D3000982EF701D280A580A2949FE0A9228091DD
:101D40008D028770B9F0DD20A9F0812F807F80346B
:101D500021F080E2800F883068F08091D30182FF0B
:101D600009C082E00E946E1C80918D028770CC2495
:101D7000C3948111C12CB12EB2948FE0B8228B2D67
:101D800090E08C30910508F0F5C1FC01EC56FF4F56
:101D90000C942935812F807F1F70882311F01295B4
:101DA000107FDD20B9F0112309F4D2C180E2800F49
:101DB000883010F0911006C090919702192B109363
:101DC000970205C090919602192B109396020E94DB
:101DD000321CBEC1802F0E94E52A112309F4CAC11A
:101DE000005E083080F1992071F110959091960273
:101DF0001923109396022AC0812F807F1F70803292
:101E000011F01295107F992029F0F1E09F1609F446
:101E100041C04FC08091D30182FD1BC0DD2069F01D
:101E2000112339F090919702192B109397020E9479
:101E3000321C80E00E94492B9DC180E00E94E52A6F
:101E4000112309F497C1812F0E942B1C0E94321C80
:101E500091C1DD2081F080919802AA2051F021E00B
:101E6000A21207C0182B181709F484C11093980206
:101E700081C1812B16C0A11003C00E94251C31C056
:101E800031E0A31609F476C1812F0E94FC290E943B
:101E9000251C70C1DD2041F085E08A1508F46AC177
:101EA000812F0E94032A66C194E09A1508F462C14A
:101EB00018C0DD2049F0AA2099F3F701858180FF41
:101EC00047C18F708583ECCFAA2059F0093309F000
:101ED0004EC1FFEF27EE33E0F15020403040E1F7F4
:101EE00044C1812F0E94FC2945C1812F869586958A
:101EF000837019F0813059F03DC1DD2019F0C8011F
:101F0000937002C080E090E00E94AD2739C1DD20CF
:101F100019F0C801937002C080E090E00E94882709
:101F20002FC16D2D802F0E940D2A2AC1812F837011
:101F300009F041C0D11022C1302F3295369537704B
:101F4000330F330F802F8F7090E0032E02C0880F65
:101F5000991F0A94E2F704FF0BC04FE050E002C063
:101F6000440F551F3A95E2F79A012095309502C02B
:101F700020E030E0169516951370123099F068F451
:101F80004091990250919A02113029F0822B932BA3
:101F90008423952304C0842B952B822B932B0E94A2
:101FA0009929ECC0822B932B2091990230919A02AF
:101FB00082279327F4CFDD2019F0812F817001C093
:101FC0008695882309F4DAC0302F3295369537701C
:101FD000330F330F802F8F7090E0032E02C0880FD5
:101FE000991F0A94E2F704FF0BC04FE050E002C0D3
:101FF000440F551F3A95E2F79A012095309502C09B
:1020000020E030E0169516951370123079F0B8F490
:102010004091E7025091E802113029F0822B932B76
:10202000842395230EC0842B952B09C0822B932BE0
:102030002091E7023091E8028227932702C0822B89
:10204000932B0E9472299AC01F70DD2039F0812FD6
:102050000E948929802F0E94032A90C0802F0E940D
:10206000FC29812F0E94772989C0802F92EF991631
:10207000A1F1991538F0E0EF9E1659F0F1EF9F1697
:1020800039F162C023EF921679F134EF9316E1F043
:102090005BC0DD20A1F084E08A1508F46BC01F71DD
:1020A00081E090E0012E02C0880F991F0A94E2F7A8
:1020B0002091E7023091E8028227932723C095E020
:1020C0009A1508F457C0EBCF8091D30182FD1DC053
:1020D000DD2029F0812F8F712AC0DD20D9F3812FD7
:1020E0008F710E94772946C0DD2051F01F7181E079
:1020F00090E0012E02C0880F991F0A94E2F702C0F7
:1021000080E090E00E94722935C0DD2099F01F71B7
:10211000812F0E9489298091D30182FF07C0E8E0C6
:102120001E9FC0011124836080938D02812F0E9425
:10213000892920C081E00E946E1CF1E0FA15D0F4DC
:1021400082E00E946E1C16C0DD2021F0AA2011F250
:10215000802F70CEAA2019F2893349F42FEF37EE81
:1021600083E0215030408040E1F700C00000802F24
:102170000E94E52A88EF8B0D843010F40E94D2274C
:10218000CC2009F48AC080918D0280FD86C0F701C1
:1021900012828595859585950E948929C7010E949F
:1021A000770B80918D028595859585950E9477297D
:1021B00074C0809197028A7A91E009F490E090933C
:1021C000E701811112C069E28DE492E00E946E275E
:1021D00009C08091E70181115EC069E28DE492E05F
:1021E0000E9461270E94321CF5CB65E3EDCFE056DB
:1021F000FF4F0C9429359091B80281E08927809394
:10220000B8021092140180913F03816080933F03D4
:10221000E1CB45E053E360E173E32CC040E153E3DD
:1022200065E073E327C046ED52E361EE72E322C03E
:1022300041EE52E366ED72E31DC04AEB52E368ECF7
:1022400072E318C048EC52E36AEB72E313C04EE944
:1022500052E36CEA72E30EC04CEA52E36EE972E3B9
:1022600009C049ED50E367EE70E304C047EE50E368
:1022700069ED70E30E942832ADCB61E081E008C0D7
:1022800061E085E005C061E08DE002C061E082E1CF
:102290000E94EC329FCB65E3A1CF2D96E2E10C9436
:1022A0005235A3E0B0E0E7E5F1E10C943635782E45
:1022B0008091130187110DC02091B802237030E086
:1022C0004091120150E081E02417350719F480E0B5
:1022D00001C081E0817080930F018091BD029091D7
:1022E0000E01981739F080930E0140E060E080E025
:1022F0000E94D92E86E1781257C08CED9CE20E9494
:10230000FE1F0EC0371508F40EC245E0741609F41E
:10231000BCC156E07512ADC184EE9DE20E94B61FAD
:1023200089832DC0971508F40CC2A4E07A1609F42D
:102330004FC0A71508F4A3C1B1E07B1295C020914E
:102340000D01220F220F29832C5F2A83253110F0E3
:1023500034E13A836091B9027091BA028091BB0274
:102360000E94CB2F162F072FF82E89819A8189176B
:1023700008F487C0A1E0A983943108F080C080915F
:102380000D018F5F80930D01598151111DC782E0AE
:102390008093140180910F01811116C7711014C729
:1023A00083E08093140110C7871508F40AC29AE0ED
:1023B0007912B8CF83E89EE208C0B71508F4D5C1FA
:1023C000EBE07E12CCC187E69EE20E945120A8CFAE
:1023D00030910D01330F330F39833C5F3A83353130
:1023E00010F044E14A83E090BA02D090BB02209101
:1023F000BC0280E4F82E5F2D529F512D1124F52E42
:10240000A981BA81AB1750F58981082F10E0F80136
:10241000E858FE4F90AD80910E018923D9F0F80164
:10242000EE0FFF1FE857FE4F6081F69EB0011124AA
:10243000B5E075956795BA95E1F78091B902680F97
:102440007E2D8D2D0E94CB2F462F282F672FC80160
:102450000E94DC2E99819F5F9983D2CFE1E0E983CE
:10246000B43108F48CCF0BC07B1608F580910F01B6
:10247000882329F040E060E080E00E94D92E198294
:102480007ECF4981E42FF0E0DF01A858BE4FD896F7
:102490008C9190910E01982331F02F2D412F602FB8
:1024A000CF010E94DC2E59815F5F59835ECFE0919E
:1024B0000D01E983F2E07F1246C0B981BB0FBB0F6B
:1024C000B983BC5FBA83B53110F0E4E1EA830091CF
:1024D000BA021091BB02F090B9026F2D702F812FBC
:1024E0000E94CB2FE62ED72EC82E6091BC026F0D16
:1024F000702F812F0E94CB2F162F072FF82E398196
:102500004A813417D0F4F9818F2F90E0FC01E8580C
:10251000FE4F30AD20910E01232359F030FF04C04F
:102520002F2D412F602F03C02C2D4E2D6D2D0E947D
:10253000DC2E29812F5F2983E2CF51E0598344317A
:1025400008F41DCF9CCF23E0721293C08981880FBD
:10255000880F89838C5F8A83853110F094E19A8398
:102560000091BA02D090BB022091BC0210E4129FED
:10257000112D1124E981FA81EF1708F067C0A981B4
:10258000EA2EF12CF701E858FE4F90AD80910E0134
:102590008923B9F0F701EE0FFF1FE858FE4F81893C
:1025A00082958F706091B902819F600D1124702F08
:1025B0008D2D0E94CB2F462F282F672FC7010E94F9
:1025C000DC2EB981BF5FB983D5CFB71508F45AC5E2
:1025D000ECE17E1609F4FDC0E71508F41EC2F9E12E
:1025E0007F123AC080910D01880F880F89838C5F1C
:1025F0008A83853110F094E19A830091BA02109198
:10260000BB02F090B9026091BC0266956695669532
:102610008091B4029091B5020E94AE2F0E94FA2ED2
:10262000805887FD8195880F682F2CE0629F612D6F
:1026300011246F0D702F812F0E94CB2F162F072F83
:10264000F82EE981FA81EF1708F43BC121E02983D4
:10265000F43108F494CE13CFF71508F4D2C1809169
:102660000F0127E1721609F442C138E1731609F42B
:1026700084C180910D018F5F80930D0188CE37E07A
:10268000731240CE88EB9DE249CEF0910D01FF0F11
:10269000FF0FF983FC5FFA83F53110F024E12A8300
:1026A0000091B9021091BA02F090BB026091BC0295
:1026B0006695669566958091B4029091B5020E94E8
:1026C000AE2F0E94FA2E805887FD8195880F382FF3
:1026D0004F2D349F312D1124832FB8010E94CB2F11
:1026E000162F072FF82E9981AA819A17B0F45981D5
:1026F000E52FF0E0DF01A858BE4FD8968C9190915D
:102700000E01982331F02F2D412F602FCF010E9411
:10271000DC2E89818F5F8983E6CFB1E0B983A43154
:1027200008F42DCEACCE88E0781203C08CEB9EE28C
:1027300005C099E079129DCF8EE99EE20E94CB20E0
:10274000EFCDA0E17A1203C08AE79DE23ECEA71545
:10275000C0F0BDE07B1231CE8DEA9DE2DFCDFCE022
:102760007F1287CF86EB9DE2D9CD2EE0721203C097
:1027700084EA9DE2D3CD3FE073127BCF89E89DE2EE
:10278000CDCD43E1741203C082E49EE21ECE471514
:1027900060F051E1751203C085E89FE2CFCF82E17E
:1027A000781267CF86E59EE2C9CF94E1791203C023
:1027B0008CE49DE2A4CDA5E17A125BCF8AE19DE293
:1027C0009ECDB2E27B1201CF8EEB9CE20E94491FAC
:1027D000A7CD10910D01110F110F1C5F4091B40294
:1027E0005091B5026091B6027091B7028091E801F4
:1027F0009091E901A091EA01B091EB01841795074E
:10280000A607B70708F057C00E943F2F082F0E9465
:102810003F2F94E1891BF0F7890F482F50E05B832D
:102820004A83FA01E858FE4F90910E0180AD89234A
:1028300009F441C001FF04C020E040E060E013C0A3
:102840000E943F2F082F0E943F2F8695782F2FE759
:10285000720F08F47FEF602F8091BB020E94CB2F94
:10286000462F282F672F8A819B810E94DC2E209182
:10287000BC0230E1230F08F42FEF60E1822F90E0DB
:102880000E94AE2FBC0184EF91E00E94013580913F
:10289000B4029091B502A091B602B091B702860F32
:1028A000971FA11DB11D8093E8019093E901A093AA
:1028B000EA01B093EB0151E05983143108F45FCD84
:1028C000DECDA981EA2FF0E0DF01A858BE4FD896EF
:1028D0008C9190910E01982331F02F2D412F602F74
:1028E000CF010E94DC2EB981BF5FB983AACEE091EF
:1028F0000D01EE0FEE0FE9831E2F1C5F153108F05E
:1029000014E181111EC06091BC0220E1620F08F445
:102910006FEF8091B4029091B5020E94AE2F6AE0F1
:1029200070E00E940135892B29F50E943F2F64E158
:102930000E94F53460910E01892F90E00E9453327D
:1029400019C03981232F30E03B832A83E12EF12CFB
:102950008A819B818E159F056CF460910E018A819E
:102960009B810E9453324A815B814F5F5F4F5B8343
:102970004A83EECF91E09983A0CF81111EC0609170
:10298000BC0220E1620F08F46FEF8091B4029091D5
:10299000B5020E94AE2F65E070E00E940135892BE0
:1029A00009F06DCD0E94303464E170E00E9415356D
:1029B00060910E010E942F3262CDA0910D01AA0FED
:1029C000AA0FA9831A2F1C5F153108F014E1F981B1
:1029D000EF2FF0E0FB83EA83E12EF12C4A815B814B
:1029E0004E155F050CF067CF60910E018A819B81C7
:1029F0000E942F322A813B812F5F3F4F3B832A83E6
:102A0000EDCF4AE1741203C08BE19FE287CC5BE11A
:102A100075122FCE8BEC9CE281CC8FE17812AAC08C
:102A200040900D01440C440CB4E05B2E540CF4E1D6
:102A3000F51510F4A4E15A2E80910F01882361F05E
:102A400040E060E080E00E94D92E80E1EDE3F2E01A
:102A5000DF011D928A95E9F780910D01811115C062
:102A60008091390290913A020E94112721E0893128
:102A7000910508F420E020933802499730F00E9435
:102A80002C2790933A02809339020DE312E078E705
:102A9000A72E71E0B72EE9E48E2EE2E09E2E312CB7
:102AA000FAEA2F2E6801E12CF12CF501EE0DFF1D45
:102AB000B081B983B41508F43FC0B51508F03CC027
:102AC0003394EB2FF0E0FB83EA83E858FE4F90ADA0
:102AD00080910E01892309F42FC0D6016C90362D08
:102AE00025E5321B08F430E07091BA02222D462D04
:102AF000240F08F42FEF4091BB0252E0259F200DD8
:102B000011242E5F249F212D1124622D631B822FFF
:102B10000E94CB2F462F282F672F8A819B810E94EE
:102B2000DC2E80913802882339F0262D31E0231BDA
:102B300008F420E0D6012C93BFEFEB1AFB0AEFEF6D
:102B4000CE1ADE0AF4E0EF16F10409F0AECF8016DB
:102B5000910649F00C5F1F4F24E0A20EB11C33E038
:102B6000331508F09FCF41E0498353E1551508F034
:102B700006CC85CC871508F4B4C19DE17912F1C06B
:102B8000409128025091290260912A0270912B02F3
:102B90008091B4029091B502A091B602B091B702B3
:102BA00084179507A607B70708F469CC80910F0131
:102BB00081110CC080910D01880F880F8983082F27
:102BC0000C5F053108F45FC004E15DC040E060E0E7
:102BD00080E00E94D92E0CEE11E01B821A82FFE7E2
:102BE000DF2E0E943F2F81FF08C0D8011C92119652
:102BF0001C92119712961C9220C00E943F2FC82E43
:102C00000E943F2F8695782F2D2D720F08F47FEFAD
:102C10008A819B81880F991F4A815B81840F951F50
:102C2000DC01A451BE4F7D016C2D8091BB020E943E
:102C3000CB2FF7016083718382832A813B812F5FD1
:102C40003F4F3B832A830D5F1F4F2431310549F6E7
:102C5000B1CF3981832F90E0FC01E858FE4F30ADB1
:102C600020910E01232361F0FC01EE0FFF1FE80FFE
:102C7000F91FE451FE4F2281408161810E94DC2EC8
:102C800049814F5F49835981501718F381E0898347
:102C9000043108F01982043108F471CB20E010E00F
:102CA00001501109822F90E080179107CCF4AC01FC
:102CB000440F551F480F591F44515E4F0196FC01A8
:102CC000EE0FFF1F8E0F9F1FFC01E451FE4F80810E
:102CD0009181A281FA0180839183A2832F5FE2CF49
:102CE0000E943F2F7801EE0CFF1C81FF09C00E0DE2
:102CF0001F1DF801E451FE4F10821182128218C08C
:102D00000E943F2F8A830E943F2F8695782F2FE7BE
:102D1000720F08F47FEF0E0D1F1D04511E4F6A81C4
:102D20008091BB020E94CB2FD8016D937D938C9331
:102D30000E94B82F0091B4021091B5022091B60202
:102D40003091B702DC01CB01800F911FA21FB31F8E
:102D50008093280290932902A0932A02B0932B0219
:102D60000ECBAEE17A1285CC80910F01882329F039
:102D700040E060E080E00E94D92E80910D01880F34
:102D8000880F94E0F92EF80E4091B4025091B502EC
:102D90006091B6027091B702809134029091350231
:102DA000A0913602B091370284179507A607B7079E
:102DB00008F090C06091B9027091BA028091BB0294
:102DC0000E94CB2FE62ED72EC82E0CE212E0E8E7A9
:102DD000F1E0FB83EA8388E8A82E81E0B82ED801D1
:102DE0008C91882381F0AA81BB818C912C2D4E2D52
:102DF0006D2D90E00E94DC2EEA81FB8183812C2DD9
:102E00004E2D6D2D0FC0AA81BB818C9120E040E03A
:102E100060E090E00E94DC2EEA81FB81838120E06B
:102E200040E060E090E00E94DC2ED80111968C9189
:102E300011978C93EA81FB81882379F081812C2D75
:102E40004E2D6D2D90E00E94DC2EAA81BB81129642
:102E50008C912C2D4E2D6D2D0EC0818120E040E0F7
:102E600060E090E00E94DC2EAA81BB8112968C91DA
:102E700020E040E060E090E00E94DC2E0E943F2FC6
:102E8000837091E009F090E0F80191830E5F1F4F8D
:102E90002A813B812C5F3F4F3B832A83A216B306D6
:102EA00009F09DCF0E94B82F0091B4021091B50295
:102EB0002091B6023091B702DC01CB01800F911F47
:102EC000A21FB31F8093340290933502A093360261
:102ED000B0933702B1E0B983E3E1EF1508F04FCAD0
:102EE000CECAB0E27B12C8C06090BB02A3E06A9E6B
:102EF000C001112496958795969587959B838A8323
:102F0000BA81B983462C512C8FEF90E0B2010E9418
:102F10001535362E80910F01882371F040E060E076
:102F200080E00E94D92E80E1EDE3F2E0DF011D9206
:102F30008A95E9F710923C0280913B028F5F809363
:102F40003B0238E7A32E31E0B32E41E4842E42E069
:102F5000942E5DE3E52E52E0F52EEA81FB814E1AB8
:102F60005F0A87016501212C21100CC080913C0271
:102F7000811108C00E943034853595401CF4D7017A
:102F80006C920CC0F8018081882341F0861530F4E2
:102F900090913B02391202C081508083D601EC919E
:102FA000EF3F29F1D8012C91F0E0B981B21790F4EC
:102FB00030E04A815B81241B350B249FC001259F93
:102FC000900D349F900D1124B2010E940135262FDF
:102FD000462D0AC0629EC00111246A817B810E9435
:102FE0000135462F20E060E0CF010E94DC2E2394C3
:102FF00054E0C50ED11C0C5F1F4F84E02812B4CFE3
:103000009FEFE91AF90AAFEFAA1ABA0A8E149F04C1
:1030100009F0A7CF80913B02381202C010923B0208
:1030200080913C028F5F8D3118F480933C0227CA57
:1030300010923C0225E432E083E09FEF960DADE371
:10304000B2E0F901833041F41C964C911C97641254
:1030500003C01C969C931C974081461510F09083EA
:103060006482319611968A169B0661F7815024502E
:1030700031098111E4CF03CAE1E27E12FACA84EC7D
:103080009CE2A4CBF8E27F120CC06BE37CE205C0AB
:1030900044E27412EECA65EA7CE280E00E94AC1E53
:1030A0003FC9F71508F432C025E272120BC08091B7
:1030B000BE0221E0482F421B08F440E0842F6DE659
:1030C0007CE2ECCF271570F033E27312E1CF8091F0
:1030D000BE0221E0382F321B08F430E0832F65EA6E
:1030E0007CE2DCCF56E2751203C06DE67CE2D5CF00
:1030F00087E27812BECA8091BE0221E0582F521B8F
:1031000008F450E0852F6BE37CE2C8CF9BE2791294
:103110000BC08091BE0221E0482F421B08F440E022
:10312000842F6DE07CE2BACF9715A0F0A9E27A1265
:103130000BC08091BE0221E0382F321B08F430E032
:10314000832F63E27CE2AACFBAE27B1292CA63E2E7
:103150007CE2A3CFECE27E1203C06DE07CE29DCF67
:10316000FFEF7F1286CA8091B4029091B502A091C0
:10317000B602B091B70288279C70AA27BB272AE025
:10318000B695A795979587952A95D1F782309105A1
:10319000A105B10571F083309105A105B10569F074
:1031A00040E00197A105B10511F060E008C064E1BD
:1031B00002C044E160E080E003C044E164E184E1F6
:1031C0000E94D92E82E0EDC82396E2E10C9452359C
:1031D00080E008959091D20192FF0DC0282F2871B0
:1031E000283019F4877F846006C0282F247124308A
:1031F00011F48B7F886093FF0DC0282F2871283130
:1032000019F4877E846106C0282F2471243111F4BB
:103210008B7E88612091D30120FF0DC0382F38713B
:10322000383019F4877F816006C0382F3171313012
:1032300011F48E7F886021FF0DC0282F287128315E
:1032400019F4877E816106C0282F2171213111F484
:103250008E7E886194FD877E0895F894E82FE2952C
:10326000EF70F0E031A1282F2F7081E090E001C0D5
:10327000880F2A95EAF7982F9095932391A392A10E
:10328000892B82A378940895A4E0B0E0EAE4F9E100
:103290000C943D3519821A821B821C8208E111E0D0
:1032A000AE014F5F5F4F7A015A01CC24C394D12CF9
:1032B000F80180818F3F09F441C0F894E82FE2952E
:1032C000EF70F0E021A18F70A60102C0440F551FDE
:1032D0008A95E2F7CA01922F982B91A392A180952B
:1032E000892382A3789400C0ECE1F1E0912C31E0D5
:1032F00021912F3F89F0A22FA295AF70B0E0909658
:103300008C9190E02F7002C0959587952A95E2F7F1
:1033100080FD02C0832F01C080E0982A330F51E066
:10332000E032F50729F7F80180818F3F11F00E9404
:103330002D19F0EAFA95F1F7F70190820F5F1F4F10
:10334000FFEFEF1AFF0A41E00C31140709F0B0CF8C
:1033500044E050E0B5018EEC91E00E946D35892B80
:10336000A9F089819A81AB81BC818093CE01909331
:10337000CF01A093D001B093D10181E080939D0251
:103380000E942C2790939C0280939B0280919D0227
:10339000811102C080E027C080919B0290919C0225
:1033A0000E9411270597B0F344E050E06EEC71E005
:1033B00083EE91E00E946D35892B91F08091CE01D2
:1033C0009091CF01A091D001B091D1018093E30100
:1033D0009093E401A093E501B093E60181E001C080
:1033E00080E010929D022496EBE00C9459357430E5
:1033F00048F46430C8F48A30B8F4462F672F0E942E
:10340000AD3108957D3F31F4623070F48A3060F45C
:1034100041E007C07C3F41F4623030F48A3020F450
:1034200040E00E944D31089580E090E00895CF93F0
:10343000DF938238910569F1B0F48133910509F485
:1034400077C048F48932910509F469C08A32910540
:1034500009F473C092C08533910509F45BC08933C8
:103460009105B9F08AC0833E910591F138F4803E10
:103470009105D1F0823E910531F17FC0863E9105E4
:10348000D9F1873E9105E9F1843E910509F075C0B7
:1034900028C02091D20120FD5BC021FD59C02091A0
:1034A000D30123FD61C069C08091D20180FD4AC073
:1034B0008091D30180FF4CC08091D20184FD50C126
:1034C00083EE90E04FC18091D20182FF3EC0F4CFE5
:1034D0008091D20182FD39C08091D30180FD38C036
:1034E000EBCF8091D30181FF39C08091D20184FD5F
:1034F00037C187EE90E036C18091D20183FF2BC0A7
:10350000F4CF8091D20183FD26C08091D30181FD4B
:1035100025C0EBCF8091D20185FD26C022C08091CD
:10352000D20185FD1EC08091D30183FF1DC00AC05A
:103530008091D20186FD1BC01DC08091D20186FD05
:1035400019C015C089E390E00DC182EE90E00AC178
:1035500080EE90E007C186EE90E004C184EE90E03A
:1035600001C185E390E0FEC089E290E0FBC08AE201
:1035700090E0F8C081E390E0F5C0EC01811530E502
:10358000930708F053C0811560E4960720F0CE0140
:103590009F70906AE7C0803E910588F58D3C91054B
:1035A00018F0CE019065DEC0883A9105C0F4853AE6
:1035B000910550F08C2F855AC82FD0E0CC5CDE4F9F
:1035C000888190E09064CEC08130910509F4C5C037
:1035D00008F4C6C0049708F4C3C0CE01C3C0813C40
:1035E000910508F0BDC08C2F885AC82FD0E0CC0FB1
:1035F000DD1FC95CDE4F888199819464B3C0811559
:10360000904258F08D2F8F710E94EA18282F2F7149
:10361000CE0199279062922BA5C0C11581E0D807F1
:10362000E0F6C83ED10508F09BC0D7CFC03692E582
:10363000D90708F053C0C03422E5D207B8F08C2F68
:103640008F718695869570E2879FA00111248C2F3B
:10365000837021E030E0B90102C0660F771F8A95C0
:10366000E2F7CB019C68842B952B7CC0C03232E5FD
:10367000D30740F08C2F8F7190E0982F8827816FAF
:10368000906A70C0C11562E5D607B0F08C2F8695A0
:10369000869520E2829FA00111248C2F837021E067
:1036A00030E0B90102C0660F771F8A95E2F7CB01BF
:1036B000842B952B9D6856C08C2F8F710E94EA1821
:1036C00095E0D695C7959A95E1F7CF70D0E0DC2FBD
:1036D000CC27D0699E01282BC90144C0C03A72E5AD
:1036E000D70708F58C2F8F71C03892E5D907A8F459
:1036F0008695869570E2879F900111248C2F8370A8
:1037000041E050E0BA0102C0660F771F8A95E2F7E8
:10371000CB019A68822B932B25C090E0982F8827A5
:10372000846F906A1FC0C03C22E5D20750F48C2FF2
:103730008F710E94EA188F7190E0982F882790620D
:1037400011C0C03E32E5D30758F4CE018F719927DE
:10375000982F8827806F906A05C081E090E002C0B2
:1037600080E090E0DF91CF91089580E090E00E94AA
:103770005834873E9E4F19F40E940F32089580E01E
:10378000089567EE7EEF80E090E00E948C3460E068
:1037900082E090E00E946E3460E083E090E00E945E
:1037A0006E3410929A021092990260E074E184E003
:1037B00090E00E948C3460E086E090E00E946E34DD
:1037C0006FEF87E090E00E946E3440E050E0BA0175
:1037D00088E090E00E94803460E08DE090E00E94FC
:1037E0006E3440E050E0BA0188E190E00E948034FD
:1037F00060E087E190E00E946E3440E050E0BA0162
:103800008CE190E00E94803460E070E080E290E023
:103810000E948C3440E050E0BA0188E190E00E94C0
:10382000803480E00E94E0310E94FF3140E050E0AF
:10383000BA018FE090E00E94803440E050E0BA018D
:1038400083E190E00E948034089580919802811174
:103850001092980208958095909197028923809301
:10386000970208959091970280919602982B9093D9
:103870004D0280919802882389F0892B80934D0214
:10388000EFE4F2E097E080E0915029F021912223CB
:10389000D9F38F5FF9CF81110E94251C48E050E0D9
:1038A0006EE872E08DE492E00E946D35892BA9F0FC
:1038B00088E0EDE4F2E0AEE8B2E001900D928A9586
:1038C000E1F7E091EE02F091EF02309731F00280E3
:1038D000F381E02D8DE492E00995089520918D0209
:1038E0008095822380938D02982F977099F430E011
:1038F000482F082E000C550B2417350759F09091CE
:10390000D30192FF07C08595859585950E947729FB
:1039100010928D0208959091D30192FB222720F9F5
:10392000281779F080FB92F99093D3016091D2012E
:103930007091D30184E090E00E948C3482E00E9478
:103940006E1C089580918C0290915B02891719F08A
:103950008F5F8770FBCF08950F931F93CF93DF93F3
:1039600080915A0282958F7009F05AC08091570257
:10397000882309F455C080918C0210915B026091FC
:10398000550270915602C0915802D091590291E0AF
:103990006F3F09F090E0292F06E0811709F440C03D
:1039A000209721F07F3F21F030E003C031E001C0DB
:1039B000322F90E030FD31C0089FF001099FF00DDB
:1039C0001124DF01A45ABD4F11963C911197371372
:1039D00024C03C91361321C012963C9112973111AC
:1039E0001CC013964D915C9114974C1B5D0B483C89
:1039F000510598F480915A028F70806180935A0229
:103A0000EF59FD4F80818F708061808385E592E062
:103A10000E94770B0E94A21C03C001968770BDCF45
:103A2000DF91CF911F910F910895A1E1B0E0EBE1FB
:103A3000FDE10C943D358C0185E0F801DE011D9619
:103A400001900D928A95E1F7F801E280909155027C
:103A5000609156024091580250915902411551050A
:103A600031F06F3F31F481E09F3F19F403C081E0F2
:103A700001C080E0F82FF1709F2E80FD1BC1F8017E
:103A800030812181C380D48085E5A82E82E0B82EC4
:103A9000F0905702F601E41BF50BFF2009F4C7C0B4
:103AA00080915A02E83CF10508F092C0482F407F0F
:103AB00009F051C0621311C093130FC0FE2CE11026
:103AC0000CC08F70806180935A02C5010E94770BF1
:103AD00080915A02F80185832AC1C114D10431F0C2
:103AE0002F3F31F481E03F3F19F403C081E001C072
:103AF00080E080FD03C081E08E2502C080E090E080
:103B0000F82FF170FF2E80FF1CC080918C02409135
:103B10005B0256E0841709F4E8C090E0589FF0017A
:103B2000599FF00D1124E45AFD4F6181261306C000
:103B30006081631303C06281E61203C0019687703F
:103B4000E9CFFE2CEE2009F4F2C080915A02816088
:103B500080935A0249C0621306C0931304C0E11057
:103B600002C0F80186C0C8010E949E29882351F135
:103B7000EE2041F120915A02822F82958F7090E0C1
:103B8000029774F0809155029091560298878F8326
:103B90001986DB86CA862C87CE0107960E94770B92
:103BA00086E0F801A5E5B2E001900D928A95E1F773
:103BB0000E94AC1C0AC06217C9F0C8010E949E296D
:103BC00081111EC0C8010E94770BFF24F394AFC07F
:103BD000482F407F81F785E592E00E94770B86E0D1
:103BE000F50111928A95E9F7F12CA1C09313E5CF65
:103BF000E110E3CFF8018583C8010E94770B54C020
:103C0000EE2001F320915A02822F82958F7090E06E
:103C1000029734F280915502909156029A838983DB
:103C20001B82DD82CC822E83CE010196B7CFE83C89
:103C3000F105D0F5FE2CEE2029F2621327C0931374
:103C400025C020915A0220FD18C0822F82958F70C6
:103C5000482F50E04115510581F0F80125834F3080
:103C6000510541F08F5F982F9295907F822F8F7032
:103C7000892B8583C8010E94770B86E0F801A5E5B2
:103C8000B2E001900D928A95E1F751C0C8010E94FF
:103C90009E29811185CF80915A02816080935A02BA
:103CA000C8010E94770B43C086E0F50111928A9506
:103CB000E9F73DC0EE2009F485CFC8010E949E2996
:103CC000F82E882309F47ECF86E0F801A5E5B2E05E
:103CD00001900D928A95E1F78091550290915602DC
:103CE0000E9432290E94AC1C22C03D872E878D8500
:103CF0009E850E943229292F22952F70223028F488
:103D00009F7039F0811105C00BC0243028F49F70DA
:103D100049F4805E883020F0C8010E94770B9F2C08
:103D2000F92C05C0F8019581907F99F7F9CF8F2D77
:103D30006196EBE00C9459358091E7029091E8028E
:103D40009C01267033272630310511F4886001C0AC
:103D5000877F0E9472290895A7E0B0E0E2EBFEE1C0
:103D60000C943635282E4B0120910D01220F220F85
:103D70002E83122F1C5F153108F014E13091BE0222
:103D80003983AE81A11708F07CC08E81682E712C1A
:103D9000F301E858FE4F90AD80910E01892309F49C
:103DA0006CC03090B9024090BA02522C1F82C301FD
:103DB000880F991FDC01A857BE4FBB83AA83C3019C
:103DC000880F991FFC01E757FE4FFD83EC83F981B3
:103DD0005F1608F040C0E52CF12CAA81BB81CC9085
:103DE000D12CF701E254FD4F8181C81AD108AC8172
:103DF000BD81AC90B12C8185A81AB108CC9C9001F2
:103E0000CD9C300D300D1124AA9CC001AB9C900DAF
:103E1000900D1124820F931F0E94542F082F609140
:103E2000BC0221E0620F08F46FEFF701EE0FFF1FF5
:103E3000E254FD4F818D928D0E94AE2F7C01950141
:103E4000A601632D742D8F81F4010995362E472E1E
:103E50008F835394BCCF2091BB028F81382F329F28
:103E6000312D1124832F632D742D0E94CB2F462FCB
:103E7000282F672FC3010E94DC2E8E818F5F8E83D7
